:100000000C9463000C94AA040C9483040C94D10403
:100010000C94D1040C94D1040C948B000C948B00A0
:100020000C948B000C948B000C948B000C948B0024
:100030000C948B000C948B000C948B000C948B0014
:100040000C9439040C948B000C9407040C94E10379
:100050000C948B000C948B000C948B000C948B00F4
:100060000C948B000C948B000000000024002700EF
:100070002A0000000008000201000003040700003D
:1000800000000000000000000000250028002B00F8
:1000900000000000230026002900040404040404D6
:1000A0000404020202020202030303030303010227
:1000B00004081020408001020408102001020408F6
:1000C00010204B05840711241FBECFEFD8E0DEBF00
:1000D000CDBF12E0A0E0B1E0ECE9FFE002C0059086
:1000E0000D92A035B107D9F723E0A0E5B2E001C039
:1000F0001D92A139B207E1F710E0C2E6D0E004C0DA
:100100002197FE010E94B607C136D107C9F70E94A8
:10011000F6050C94C1070C940000CF92DF92EF9289
:10012000FF920F931F93CF93DF936C017A018B01A2
:10013000C0E0D0E0CE15DF0589F0D8016D918D01CA
:10014000D601ED91FC910190F081E02DC601099559
:10015000892B11F47E0102C02196ECCFC701DF91FB
:10016000CF911F910F91FF90EF90DF90CF90089566
:10017000FC01538D448D252F30E0842F90E0821BAD
:10018000930B541710F0CF96089501970895FC0132
:10019000918D828D981761F0828DDF01A80FB11DBE
:1001A0005D968C91928D9F5F9F73928F90E00895E2
:1001B0008FEF9FEF0895FC01918D828D981731F09C
:1001C000828DE80FF11D858D90E008958FEF9FEFF0
:1001D0000895FC01918D228D892F90E0805C9F4FC6
:1001E000821B91098F739927089585ED92E00E94F3
:1001F000E90021E0892B09F420E0822F0895FC0119
:10020000848DDF01A80FB11DA35ABF4F2C91848D9F
:1002100090E001968F739927848FA689B7892C93D4
:10022000A089B1898C9180648C93938D848D98136F
:1002300006C00288F389E02D80818F7D8083089538
:10024000EF92FF920F931F93CF93DF93EC0181E026
:10025000888F9B8D8C8D981305C0E889F9898081E2
:1002600085FD24C0F62E0B8D10E00F5F1F4F0F731E
:100270001127E02E8C8DE8120CC00FB607FCFACFC8
:10028000E889F989808185FFF5CFCE010E94FF00C2
:10029000F1CF8B8DFE01E80FF11DE35AFF4FF08285
:1002A0000B8FEA89FB898081806207C0EE89FF8914
:1002B0006083E889F98980818064808381E090E0AF
:1002C000DF91CF911F910F91FF90EF900895CF9301
:1002D000DF93EC01888D8823C9F0EA89FB8980814E
:1002E00085FD05C0A889B9898C9186FD0FC00FB620
:1002F00007FCF5CF808185FFF2CFA889B9898C9161
:1003000085FFEDCFCE010E94FF00E7CFDF91CF91B7
:10031000089580E090E0892B29F00E94F50081117A
:100320000C9400000895833081F028F4813099F016
:100330008230A1F008958730A9F08830B9F0843078
:10034000D1F4809180008F7D03C0809180008F77F1
:1003500080938000089584B58F7702C084B58F7D27
:1003600084BD08958091B0008F7703C08091B00064
:100370008F7D8093B00008951F93CF93DF93282F34
:1003800030E0F901EE58FF4F8491F901E255FF4F3B
:10039000D491F901E656FF4FC491CC23C9F0162F32
:1003A00081110E949301EC2FF0E0EE0FFF1FEA573E
:1003B000FF4FA591B4918FB7F894111105C09C918E
:1003C000ED2FE095E92302C0EC91ED2BEC938FBF6C
:1003D000DF91CF911F910895CF93DF9390E0FC01BF
:1003E000E255FF4F2491FC01E656FF4F849188238C
:1003F00061F190E0880F991FFC01E859FF4FC5910A
:10040000D491FC01EA57FF4FA591B491611109C045
:100410009FB7F8948881209582238883EC912E23BE
:100420000BC0623061F49FB7F8943881822F8095B9
:1004300083238883EC912E2B2C939FBF06C08FB70C
:10044000F894E8812E2B28838FBFDF91CF910895F8
:100450003FB7F8948091CA029091CB02A091CC0250
:10046000B091CD0226B5A89B05C02F3F19F001968B
:10047000A11DB11D3FBFBA2FA92F982F8827820F2A
:10048000911DA11DB11DBC01CD0142E0660F771F7A
:10049000881F991F4A95D1F7089508952091D30296
:1004A0003091D4022817390771F49091D1028091CC
:1004B000D202981741F0E091D102F0E0EB57FD4FE6
:1004C000808190E008958FEF9FEF089508951F9326
:1004D000CF93DF93DC015C962D913C915D972115C4
:1004E000310539F481E090E013969C938E93129736
:1004F0003DC05196ED91FC91529750969C9150972A
:10050000892F80951FB75E964C915E9741FB7727A8
:1005100070F941FD6095F8944081772311F0492BE3
:1005200001C048234083E9012197F1F748E0508159
:1005300060FF02C0592B01C058235083E901219765
:10054000F1F76695415099F7772321F0908189233F
:10055000808303C08081982B90831FBF5C968D9110
:100560009C915D970197F1F721E030E0C901DF919F
:10057000CF911F9108952091D3023091D402281772
:10058000390771F48091D2022091D10290E0805C11
:100590009F4F821B910960E470E00E948E070895CE
:1005A00080E090E008952091D3023091D402281782
:1005B0003907B9F49091D1028091D202981789F04D
:1005C000E091D102F0E0EB57FD4F80812091D10204
:1005D00030E02F5F3F4F2F7333272093D10290E0FD
:1005E00008958FEF9FEF0895E091D302F091D40228
:1005F000E817F90769F4A389B4899C9185898095E6
:1006000089238C931092D4021092D30281E0089532
:1006100080E00895089580E090E008959091CE02E2
:100620008091CF02981761F09F5F9D3208F090E0B3
:10063000E92FF0E0EA5AFD4F80819093CE020895B1
:1006400080E0089580918402882319F0109284023A
:100650000BC080918302882319F01092830204C09A
:100660000E940E03882311F090E008958FEF9FEF12
:10067000089580918302811112C0809184028111BA
:100680000EC00E940E03882311F0982F01C090E045
:100690009093830281E0911103C080E0089581E08E
:1006A0000895CF92DF92EF92FF920F931F93CF9313
:1006B000DF932091D00230E0F901EE58FF4F849192
:1006C000F901E255FF4FD491F901E656FF4FC4916D
:1006D000CC2391F081110E949301EC2FF0E0EE0FFA
:1006E000FF1FE057FF4FA591B491EC91ED2331E04E
:1006F00009F430E0832F02C080E090E02FB7F89437
:100700004091C6025091C7026091C8027091C9021F
:100710002FBF009152021091530220915402309148
:1007200055026A017B01C01AD10AE20AF30A970155
:1007300086010B3F11052105310520F01092510271
:10074000109250024093520250935302609354020D
:1007500070935502209151023FEF320F383048F428
:1007600001C0880F3A95EAF790915002892B809347
:10077000500281E0820F809351028B30B9F4809156
:10078000CF028F5F8D3208F080E09091CE02891702
:1007900049F0E82FF0E090915002EA5AFD4F908323
:1007A0008093CF021092510210925002DF91CF91AC
:1007B0001F910F91FF90EF90DF90CF9008950E94CE
:1007C000BC071F920F920FB60F9211242F933F93E5
:1007D0004F935F936F937F938F939F93AF93BF9349
:1007E000EF93FF9385ED92E00E94FF00FF91EF9160
:1007F000BF91AF919F918F917F916F915F914F9139
:100800003F912F910F900FBE0F901F9018951F9240
:100810000F920FB60F9211242F938F939F93EF9304
:10082000FF93E091E502F091E6028081E091EB0216
:10083000F091EC0282FD12C090818091EE028F5FF8
:100840008F732091EF02821751F0E091EE02F0E0F9
:10085000EB52FD4F958F8093EE0201C08081FF9196
:10086000EF919F918F912F910F900FBE0F901F903E
:1008700018951F920F920FB60F9211242F933F934A
:100880008F939F93AF93BF938091C6029091C702BD
:10089000A091C802B091C9023091C50223E0230F94
:1008A0002D3720F40196A11DB11D05C026E8230FA8
:1008B0000296A11DB11D2093C5028093C60290939C
:1008C000C702A093C802B093C9028091CA02909156
:1008D000CB02A091CC02B091CD020196A11DB11D19
:1008E0008093CA029093CB02A093CC02B093CD0226
:1008F000BF91AF919F918F913F912F910F900FBE1C
:100900000F901F9018951F920F920FB60F921124FF
:100910002F933F934F935F936F937F938F939F9307
:10092000AF93BF93EF93FF93E0910201F091030126
:100930000995FF91EF91BF91AF919F918F917F9119
:100940006F915F914F913F912F910F900FBE0F903C
:100950001F9018951F920F920FB60F9211242F938C
:100960003F934F935F936F937F938F939F93AF9337
:10097000BF93EF93FF93E0910001F091010109957E
:10098000FF91EF91BF91AF919F918F917F916F9167
:100990005F914F913F912F910F900FBE0F901F903D
:1009A00018951F920F920FB60F9211242F933F9319
:1009B0004F935F936F937F938F939F93AF93BF9367
:1009C000EF93FF93E091D302F091D402309709F4B2
:1009D00051C0968DA685B785858591FF04C09C91F1
:1009E000892329F447C09C91892309F043C0A38936
:1009F000B4899C918589809589238C938689978970
:100A00000197F1F7608D718DA685B785558538E022
:100A100020E0CB010197F1F7822F90E09595879523
:100A2000282F4C91452309F02068315091F7868D8D
:100A300081FD20958091D20290E001968F739927D5
:100A40003091D102381749F0A091D202B0E0AB57F3
:100A5000BD4F2C938093D20203C0868D8160868F18
:100A6000828D938D0197F1F7A389B4899C91858933
:100A7000892B8C93FF91EF91BF91AF919F918F91B3
:100A80007F916F915F914F913F912F910F900FBE8A
:100A90000F901F9018951092D8021092D70288EEEE
:100AA00093E0A0E0B0E08093D9029093DA02A093A3
:100AB000DB02B093DC022BEE31E03093D6022093C0
:100AC000D50225EC30E03093E2022093E10224ECE1
:100AD00030E03093E4022093E30220EC30E03093E6
:100AE000E6022093E50221EC30E03093E802209307
:100AF000E70222EC30E03093EA022093E90226EC90
:100B000030E03093EC022093EB021092EE02109250
:100B1000EF021092F0021092F102109275031092FF
:100B200074038093760390937703A0937803B09334
:100B300079038DEF91E09093730380937203109289
:100B400089031092880310928B0310928A031092EB
:100B50008D0310928C0310928F0310928E0360917C
:100B600090036E7F6260609390036695617081E090
:100B700068278BE00E94BC0161E08BE00E94EC01E1
:100B8000E9EBF0E0E491E0938203E5EAF0E0E49140
:100B9000F0E0EE0FFF1FEA57FF4F8591949190937D
:100BA00084038093830360E08AE00E94EC018091DB
:100BB000900381FD04C061E08AE00E94BC018AE0EC
:100BC00080937E03E8EBF0E0E491E0937F03E4EAB6
:100BD000F0E0E491F0E0EE0FFF1FE057FF4F85914A
:100BE000949190938103809380030895789484B5C1
:100BF000826084BD84B5816084BD85B5826085BD19
:100C000085B5816085BD80916E00816080936E00A6
:100C10001092810080918100826080938100809198
:100C20008100816080938100809180008160809349
:100C300080008091B10084608093B1008091B00009
:100C400081608093B00080917A00846080937A0004
:100C500080917A00826080937A0080917A0081602E
:100C600080937A0080917A00806880937A00109255
:100C7000C1000E9428024B015C0188EEC82E83E06F
:100C8000D82EE12CF12C0E942802DC01CB0188191E
:100C90009909AA09BB09883E9340A105B10558F0FE
:100CA00021E0C21AD108E108F10888EE880E83E03D
:100CB000981EA11CB11CC114D104E104F10419F760
:100CC00088E08093D00262E083E00E94EC0162E061
:100CD00088E00E94EC011092CF021092CE0281E5D2
:100CE00093E0909303018093020180916900837FD8
:100CF000886080936900E99A10928D0310928C03AA
:100D000010928B0310928A03109289031092880329
:100D10008DE991E090938F0380938E0390917E03F1
:100D2000963108F057C02DEB30E0309389032093C3
:100D300088032BE931E030938B0320938A032CE264
:100D400031E030938D0320938C032091680098301C
:100D500050F031E09E3008F430E081E001C0880FAF
:100D60003A95EAF701C084E0822B809368009830BE
:100D700038F09E3040F0963148F020E030E008C076
:100D80002DE630E005C02BE630E002C02CE630E076
:100D90003093860320938503983030F481E001C0BE
:100DA000880F9A95EAF70EC0292F30E09E3018F48C
:100DB0002850310902C02E50310981E001C0880F4E
:100DC0002A95EAF78093870380918E0390918F0391
:100DD0000197F1F780918C0390918D03892B21F17C
:100DE0008091D3029091D40223E082379207E1F000
:100DF000009711F00E94F402809190038E7F8093FF
:100E000090031092D2021092D10282E793E0909365
:100E1000D4028093D302E0918503F0918603908100
:100E200080918703892B8083E091E502F091E602AF
:100E300082E08083E091E102F091E2021082E09191
:100E4000E302F091E4028FEC80831092ED02E091D6
:100E5000E902F091EA0286E08083E091E702F091F6
:100E6000E802808180618083E091E702F091E802EE
:100E7000808188608083E091E702F091E8028081C0
:100E800080688083E091E702F091E80280818F7DA5
:100E9000808340E450E06BE072E085ED92E00E94D8
:100EA0008D0042E050E06CE472E085ED92E00E943B
:100EB0008D000E943903882321F10E942203803F84
:100EC00091F40E9439038823E1F30E9422038150A8
:100ED000833EB8F4E82FF0E0EC5FFE4F60816623BC
:100EE00081F0605808C08150833E58F4E82FF0E04C
:100EF000EC5FFE4F6081662321F082E793E00E9461
:100F000067020E948901D5CF8DEF91E09093730322
:100F10008093720382E793E00C94F40297FB072E10
:100F200016F4009407D077FD09D00E94A20707FCB1
:100F300005D03EF4909581959F4F089570956195E9
:100F40007F4F0895AA1BBB1B51E107C0AA1FBB1FFF
:100F5000A617B70710F0A61BB70B881F991F5A9545
:100F6000A9F780959095BC01CD010895EE0FFF1F64
:100F70000590F491E02D099481E090E0F8940C94B0
:100F8000C10710E0C2E6D0E004C0FE010E94B6072F
:0C0F90002196C336D107C9F7F894FFCFB3
:100F9C004D024D0243003F3D3B3C58004442403E15
:100FAC000F290000382A001D10020000002C1F1E03
:100FBC00110300002E2D201205040000392F2114DE
:100FCC0013060000313023221507000000322416CE
:100FDC0008000000332517180B0A000034352627AB
:100FEC00190C00000028001A0D00003A361C1B00DA
:100FFC00000000002B000000000E00004F004B47CB
:10100C000000005253504C4D480145574E514A3741
:10101C0049460000000041000000000000000000F4
:10102C0000000000000000000000000000000000B4
:10103C0000000000000000000000000000000000A4
:10104C000000000000000000000000000000000094
:10105C000000000000000000000000000000000084
:10106C000000000000000000000000000000000074
:10107C00000000000000090000000020018D00B8F5
:10108C00006701E900C700DB000000000067028D6B
:10109C00000B036602BB02D3024E02524D204E6976
:1010AC006D627573204B6579626F617264202D20BF
:1010BC0050532F3220636F6E76657273696F6E2C8E
:1010CC00207777772E7468656E696D6275732E6301
:1010DC006F2E756B20283230313829000D0A000034
:00000001FF
